:02000000632873
:0800080005280B181B288B18BA
:100010000A2808000B1206088B109B210608AB006B
:100020002B1814280330A5005B20CC3025083D0890
:100030000B168B1732288B1106080B109B21060814
:10004000AB002B08AB1B26280130A5002B082B1B6F
:100050002B280230A5005B20A5212508BA203D08E9
:100060008B158B1701303C0603191E210130250624
:10007000031D4228000001303D06031DEC2800301E
:10008000BD005A2802302506031D4E28000002300C
:100090003D06031DF3280030BD005A280330250615
:1000A000031D5A28000003303D06031DFD280030C3
:1000B000BD005A28A9289B2106090B108B15C139B0
:1000C000031908005B2800000130A600A700A80063
:1000D000B400B500B600B700B800B900BA01BB0162
:1000E0000030BC00BD0041308400FE30C1000D3046
:1000F000C2008530C3001030C4003230C50010305B
:10010000C6001030C7000030C8003D30C9000230C2
:10011000CA00850107309F008316D73086008113FF
:10012000011383128B1106080B108B158B100B1605
:1001300083129817181683161930990018159816F7
:1001400083128B171A081A081A080030AC001F30E7
:10015000AE0000008616A5218612A521A521A521A5
:10016000A521A521A521A9281430AD001430AF0088
:100170002521080099000C1EBB2808003330990087
:100180000C1EC0280800413099000C1EC528A5216E
:100190000800423099000C1ECB28A52108004330EE
:1001A00099000C1ED128A5210800443099000C1E8E
:1001B000D728A52108008500A521A52100308500AC
:1001C000A5210800820700340134023404340834C5
:1001D00010342034403480340130BD00AA3008216E
:1001E0000C30D221EC2800000230BD001921033070
:1001F000B2211E210930B221F32800000330BD00D6
:1002000019210330B2211E21A5210030BD00A928EB
:10021000000049082521A32149082521A3214908D7
:100220002521A32149082521A32149082521A3210E
:1002300008000130BC000D30252108000030BC0052
:100240000B302521080000000800AC0046214A08B8
:10025000AA009F30B2000830B000B20C03184D2144
:10026000031C5221B00B2D292C08B1000830B0001E
:10027000B10C03184D21031C5221B00B3829522117
:100280009D2197219721AA0B2929003441085A2141
:1002900042085A2143087821003444085A2145086D
:1002A0007821003446085A21470878210034173055
:1002B0005A210034A400861600000000000000004F
:1002C000000000000000000000000000000000002E
:1002D0008612000000000000000000000000000086
:1002E00000000000000000000000A40B5B290034A7
:1002F000A4008612000000000000000000000000C2
:100300000000000000000000000000008612000055
:1003100000000000000000000000000000000000DD
:10032000000000000000A40B7929003400340130E3
:10033000A6290530A6290A30A6291430A6292D3071
:10034000A6293230A6296430A629FA30A000C73089
:10035000A1000130A200A10BAE29A20BAB29A00B7A
:10036000A7290034A300FA30A000C730A100BB3099
:10037000A200A10BBC29A20BB929A00BB529A30B84
:10038000B3290034A3007D30A000C730A100BB30EA
:10039000A200A10BCC29A20BC929A00BC529A30B34
:1003A000C3290034A3000430A000C730A100BB3033
:1003B000A200A10BDC29A20BD929A00BD529A30BE4
:0403C000D329003409
:02400E00B003FD
:00000001FF
